:020000040800F2
:1000000000070020F1010008852500083D250008B3
:10001000652500083D2500085D250008F30100085E
:10002000F3010008F3010008F3010008653500083A
:10003000F3010008F3010008F3010008F3010008D0
:10004000F3010008F3010008F3010008F3010008C0
:10005000F3010008F301000899420008C1420008BA
:10006000E94200081143000839430008F301000881
:10007000F3010008F3010008F3010008F301000890
:10008000F3010008F3010008F3010008F301000880
:10009000F30100081D2500082D2500086143000814
:1000A000F3010008F3010008F3010008F301000860
:1000B00035440008F3010008F3010008F3010008CB
:1000C000F3010008F3010008F3010008F301000840
:1000D000F3010008F3010008F3010008F301000830
:1000E000C5430008F3010008F3010008F30100080C
:1000F000F3010008F3010008F3010008F301000810
:10010000F3010008F3010008F3010008F3010008FF
:10011000F3010008F3010008F3010008F3010008EF
:10012000F3010008F3010008F3010008F3010008DF
:10013000F3010008F3010008F3010008F3010008CF
:10014000F3010008F3010008F3010008F3010008BF
:10015000F3010008F3010008F3010008F3010008AF
:10016000F3010008F3010008F3010008F30100089F
:10017000F3010008F3010008F3010008F30100088F
:10018000F3010008F3010008F3010008F30100087F
:10019000F3010008F3010008F3010008F30100086F
:1001A000F3010008F3010008F3010008F30100085F
:1001B000F3010008F3010008F3010008F30100084F
:1001C000F3010008F3010008F3010008F30100083F
:1001D000F3010008F3010008F3010008F30100082F
:1001E000610F000800000000000000000000000097
:1001F00002E000F000F8FEE772B6374880F30888A6
:10020000364880F3098836483649086040F20000D5
:10021000CCF200004EF63471CEF200010860BFF35C
:100220004F8FBFF36F8F40F20000C0F2F0004EF628
:100230008851CEF200010860BFF34F8FBFF36F8F7C
:100240004FF00000E1EE100A4EF63C71CEF20001D4
:100250000860062080F31488BFF36F8F03F04CFE14
:1002600003F0DEFE4FF055301F491B4A91423CBF60
:1002700041F8040BFAE71D49184A91423CBF41F886
:10028000040BFAE71A491B4A1B4B9A423EBF51F82E
:10029000040B42F8040BF8E700201849184A914271
:1002A0003CBF41F8040BFAE703F02AFE03F0FEFE20
:1002B000144C154DAC4203DA54F8041B8847F9E797
:1002C00000F042F8114C124DAC4203DA54F8041B12
:1002D0008847F9E703F012BE000700200023002042
:1002E0000000000808ED00E00001002000070020E9
:1002F000E8460008002300207C2300208023002003
:100300001C510020E0010008E4010008E40100089D
:10031000E40100082DE9F04F2DED108AC1F80CD052
:10032000C3689D46BDEC108ABDE8F08F002383F3BF
:1003300011882846A047002003F084FAFEE703F066
:100340000DFA00DFFEE70000F8B500F01BFE03F039
:1003500075FD074603F0C6FD0546D0BB294B9F42FD
:1003600037D001339F4237D0274B27F0FF029A4204
:1003700035D1F8B200F03EFC2E4642F2107400F087
:100380003FFC08B10024264601F0B4F858B303201E
:1003900000F03EF80024264635B11C4B9F4203D0A6
:1003A00003F098FD00242646002003F051FD0EB115
:1003B00000F044F800F056FC00F0E6FD02F0EAF828
:1003C0000546B4B900F096FC4FF47A7003F040FA99
:1003D000F7E72E460024D2E704460126CFE706467B
:1003E00040F6C414CBE7002CD6D04FF47A74012623
:1003F000D2E702F0CFF8431BA342E3D900F01EF886
:10040000DCE700BF010007B0000008B0263A09B0E1
:10041000084B187003280CD8DFE800F00805020824
:10042000022000F00DBE022000F002BE024B0022AE
:100430005A607047802300208423002010B501F00B
:1004400059F830B1234B03221A70234B00225A6013
:1004500010BD224B224A1C4619680131F8D00433E2
:100460009342F9D16268A242F2D31E4B9B6803F11A
:10047000006303F510439A42EAD203F0FDFC03F057
:100480000FFD002000F09AFD0220FFF7C1FF164B80
:100490009A6D00229A65996F9A67996FD96DDA659E
:1004A000D96FDA67D96F196E1A66D3F88010C3F85E
:1004B0008020D3F8803072B64FF0E0233021C3F8AB
:1004C000084DD4E9003281F311889D4683F30888F2
:1004D0001047BDE7802300208423002000900008FF
:1004E000209000080023002000100240094A1368F1
:1004F00049F2690099B21B0C00FB01331360064BF3
:10050000186844F2506182B2000C01FB02001860CE
:1005100080B27047142300201023002010B5002162
:100520001022044600F0A6FD034B03CB206061605F
:100530001868A06010BD00BF9075FF1F2DE9F04145
:10054000ADF5507D0DF13C086EAC40F275120746DA
:100550000D4610A80021C8F8001000F08BFD4FF4E4
:10056000C4720021204600F085FD02F013F8254BEF
:100570004FF47A72B0FBF2F0186093E807000223A0
:1005800084E807000DF5ED702382FFF7C7FF4BF2FB
:1005900014531D49238406A803F0E2FF202384F8A6
:1005A00032310DF2EB2606AB0DF1380C1A4603CAB8
:1005B000624530607160134606F10806F6D1414687
:1005C0000122204600F0A2FD00230393AB7E02939C
:1005D00005F11903019380B20123CDE90480009352
:1005E000E97E06A3D3E90023384602F091FB0DF51E
:1005F000507DBDE8F08100BFAFF300809E6AC4214A
:10060000818A46EE8C230020704500082DE9F041D8
:100610002C4C237ADAB080460D465BBB27A92846CE
:1006200000F084FE0746002842D19DF89D60C82E48
:100630003ED801464FF4A662204600F01BFD4FF461
:100640008073C4F8F8314FF40073C4F80C334FF4DE
:100650004073C4F8203432460DF19E0104F10900C4
:1006600000F0F6FC26449DF89C30777223720BB99B
:10067000EB7E23728122002106AC27A800F0FAFC51
:100680000122214627A800F08DFE00230393AB7EB4
:10069000029305F1190380B201932823CDE90440A8
:1006A0000093E97E05A3D3E90023404602F030FB26
:1006B0005AB0BDE8F08100BFAFF3008026417272EE
:1006C000DF25D7B798480020F0B5254E4FF48A753E
:1006D00005FB0065F1B096F8D83085F8DC300024D1
:1006E000D822214685F8E8403AA800F0C3FC06F17C
:1006F000090000F0B7FCD5F8E4308DF8F000C2B284
:1007000006AF06F109010DF1F100CDE93A3400F030
:100710009FFC394601223AA800F070FE80B2CDE974
:10072000047008230127CDE9023706F1D8030193AD
:1007300030230093317A0B4807A3D3E9002302F05A
:10074000E7FAA04206DD01F025FFC5F8E0003846D3
:1007500071B0F0BD2046FBE778F6339F93CACD8D8C
:1007600098480020A43300202DE9F0411D4D1E4E75
:100770001E4F86B0284602F0F7FA034658B300240D
:10078000CDE90344ADF81440027B8DF8142099683C
:100790004068029403AA03C21B68DFF8548043F048
:1007A0000043029301F0F8FE821941F10003009426
:1007B00002A9384601F0B2F8A04205DD284602F051
:1007C000D7FA88F80040D5E798F80030072B05D80D
:1007D000013388F8003006B0BDE8F081014802F02E
:1007E000C7FAF8E7A433002040420F00D8330020B6
:1007F000CD4D002070B50D4614461E4602F0E4F9BA
:1008000050B9022E10D1012C0ED112A3D3E900232E
:10081000C5E90023012007E0282C10D005D8012CC1
:1008200009D0052C0FD0002070BD302CFBD10BA3BC
:10083000D3E90023ECE70BA3D3E90023E8E70BA3FC
:10084000D3E90023E4E70BA3D3E90023E0E700BFEB
:10085000AFF30080401DA12026812A0B78F6339F3C
:1008600093CACD8D9E6AC421818A46EE264172725A
:10087000DF25D7B7F017304A39059E5638B50546FB
:100880000E4C0021013500F0BBFBA4F82C55B4F848
:100890002C0500F09DFB78B1B4F82C0500F0A8FB06
:1008A000014648B9B4F82C0500F0AAFBB4F82C3581
:1008B0000133A4F82C35EAE738BD00BF9848002082
:1008C00010B50A4B0A4A1A6003F5805393F8482082
:1008D0003AB95C6C2CB1204600F08AFE204603F049
:1008E000F5FDBDE81040034800F082BED83300207B
:1008F000C4450008084400202DE9F04F8FB000AF38
:1009000005460C4602F060F9002849D1237E022BEF
:100910001BD1E38A012B18D101F03CFE0646FFF7FC
:10092000E5FD03464FF4C870DFF8C482B3FBF0F274
:1009300006F5167602FB103316FA83F3C8F800307A
:10094000E37E33B9A34B00221A703C37BD46BDE8A5
:10095000F08F07F12401204600F0A6FC0028F4D116
:1009600007F11400FFF7DAFD97F8264007F11401AC
:10097000224607F1270003F0C1FD0028E2D10F2C29
:1009800008D8944B1C70D8F80030A3F51673C8F83B
:100990000030DAE797F82410284602F00DF9D4E782
:1009A000E38A282B2BD010D8012B23D0052BCCD1B8
:1009B000BFF34F8F8849894BCA6802F4E062134342
:1009C000CB60BFF34F8F00BFFDE7302BBDD1844E0E
:1009D000E17E327A9142B8D1607E3146002291F8B0
:1009E000DC50854200F0A5800132042A01F58A71AD
:1009F000F5D1AAE721462846FFF7A0FDA5E7214645
:100A00002846FFF703FEA0E7B2F8EC507B6005F143
:100A100003094FEA99094FEA8902D11DC908A8EBD9
:100A2000C1039D46EB460021584600F023FB04F12C
:100A3000EE012A463144584600F00AFB7B6813B9A0
:100A4000012000F0BBFA96F8D20000F0C1FA04468B
:100A500030B9307200F0DCFA204600F0AFFAB1E0B5
:100A6000D6F8D4203AB996F8D200B6F82C258242AE
:100A700001D8FFF703FFD6F8D4202A44944208D2C5
:100A800096F8D200B6F82C250130824201D8FFF743
:100A9000F5FE70685FFA89F2594600F0F3FA08B97A
:100AA000C54679E0726896F8D2002A447260D6F89A
:100AB000D42005EB0209C6F8D49000F089FA8145EC
:100AC00009D396F8D220D6F8D4000132001B86F85C
:100AD000D220C6F8D400FF2D0FD80024347200F0C5
:100AE00097FA204600F06AFA00F004FD3D4B1881A9
:100AF00008B9FFF7A3FCC54627E7BB6896F8D900FD
:100B00000AFB0362FB68D2F8E41082F8E83001F5D2
:100B10008061C2F8E030C2F8E410FFF7D5FDFFF7BE
:100B200023FE96F8D920013202F0030286F8D9207C
:100B3000B6E74FF48A7A0AFB02F505F1EA0131447F
:100B4000204600F087FCF86000287FF4FEAE3544B4
:100B5000012285F8E82001F01DFDD5F8E020D6ED52
:100B6000007ADFED216A801A192838BF192040F673
:100B7000B832904228BF1046B8EE677A07EE900A66
:100B8000F8EEE77A67EEA67ADFED186AE7EE267AE6
:100B9000FCEEE77AC6ED007A96F8D930BB60BA6809
:100BA00073680AFB02F4321992F8E81059B1D2F8CE
:100BB000E4108B42E8463FF427AF002182F8E810AA
:100BC000C2F8E010C5467368064A9B0A01331381D8
:100BD000BBE600BF9D33002000ED00E00400FA05F5
:100BE000984800208C230020CDCCCC3D6666663F23
:100BF000A0330020014B1870704700BF98230020DD
:100C000038B54FF00054134B22689A4220D1124B52
:100C1000627D12481A70237D03724FF48073C0F80E
:100C2000F8314FF40073C0F80C3300254FF44073D3
:100C3000C0F820340A49C0F8E450C922093000F055
:100C400007FAE0222946204600F014FA012038BDB8
:100C50000020FCE79AAD44C5982300209848002066
:100C60001600002037B500F045FC194D19492881C0
:100C700002236B7100220123174801F07BF8002347
:100C80000193164B164900931648174B4FF48052A8
:100C900001F06AFF154B197811B1124801F08CFF71
:100CA00001F078FC0446FFF721FC4FF4C873B0FB59
:100CB000F3F202FB130304F5167010FA83F00C4BE9
:100CC000186003F00FF908B10F232B8103B030BD7A
:100CD0008C23002040420F00D8330020F507000885
:100CE0009C230020A4330020F9080008982300204A
:100CF000A03300202DE9F04F2DED028B90A7D7E90E
:100D000000670FF24429D9E90089884C95B00DADF0
:100D10009FED848BFFF728FDDFF834B200230C939E
:100D2000ADF83C300D936B6000230DF125028DED85
:100D3000008B4FF0010A09A958468DF825308DF82F
:100D400024A001F08FFB9DF824200023002A40F00E
:100D5000AF80204601F038FF0546002847D1DFF874
:100D6000F4B101F017FCDBF8003098423FD301F0FA
:100D700011FC0790FFF7BAFB079A4FF4C873B0FB5A
:100D8000F3F101FB130302F5167010FA83F0CBF8B0
:100D90000000DFF8C4B19BF800100791002914BFD0
:100DA0002B46534610A88DF83030FFF7B7FB079954
:100DB000C1F11002D2B2062A10AB28BF0622194494
:100DC0000DF13100079200F043F9079A0CAB039341
:100DD000182302930132564BD2B2CDE900A30492FC
:100DE0003B463246204601F035FF8BF8005001F0BB
:100DF000D1FB504A504D1368C31AB3F57A7F32D3F2
:100E0000106001F0C9FB02460B46204601F0BAFF14
:100E1000204601F0D9FE30B32B7ADFF840A1002B39
:100E200014BF032302238AF8053001F0B3FB0DF150
:100E3000400B4FF47A730122B0FBF3F05946CAF825
:100E40000000504600F008FA182302933B4B019330
:100E500080B240F25513CDE903B0009342464B46B1
:100E6000204601F0F7FE2B7AB3B101F093FB4FF06F
:100E7000000A83464FF48A7295F8D900504400F076
:100E8000030002FB005393F8E810002934D00AF164
:100E9000010ABAF1040FEFD1C82002F0D9FC2B7A75
:100EA000002B7FF434AF15B0BDEC028BBDE8F08FA2
:100EB0004FF0904110A84A6982F010024A61194629
:100EC000102200F0D7F80DF126030AAA0CA9584603
:100ED00000F018FE95E8030011AB83E803009DF8CD
:100EE0003C308DF84C300C9B109310A9DDE90A239F
:100EF000204602F01BF917E7D3F8E01049B12B6840
:100F0000FA2B38BFFA23ABEB01010533B1EB430FEA
:100F1000BDD3FFF7D9FB4FF48A720028B7D1BBE7E6
:100F2000AFF300800000000000000000A4330020A8
:100F30009C330020C84D002098480020CC4D002054
:100F4000401DA12026812A0BF1C6A7C1D068080F39
:100F5000D8330020A03300209D3300208C230020B4
:100F600008B5054800F074FEBDE80840034A04498E
:100F7000002003F0A5BA00BFD8330020084E00209F
:100F8000C10800087047000070B502F0FDFD094E71
:100F9000094D3080002428683388834208D902F044
:100FA000EFFD2B6804440133B4F5104F2B60F2D3EE
:100FB00070BD00BFFC4D0020D04D002002F096BE59
:100FC00000F10060920000F5104002F019BE000030
:100FD000054B1A68054B1B889B1A834202D91044A3
:100FE00002F0CEBD00207047D04D0020FC4D002007
:100FF000024B1B68184402F0C9BD00BFD04D002051
:10100000024B1B68184402F0D3BD00BFD04D002036
:10101000064991F8243033B10023086A81F824305E
:101020000822FFF7CDBF0120704700BFD44D00203C
:10103000022802BF4FF0904310229A6170470000CF
:10104000022802BF4FF090434FF480129A6170471C
:1010500010B50023934203D0CC5CC4540133F9E7AC
:1010600010BD000003460246D01A12F9011B0029E8
:10107000FAD1704702440346934202D003F8011BA1
:10108000FAE770472DE9F8431F4D144695F82420E0
:101090000746884652BBDFF870909CB395F8243021
:1010A0002BB92022FF2148462F62FFF7E3FF95F876
:1010B0002400C0F10802A24228BF2246D6B241460F
:1010C000920005EB8000FFF7C3FF95F82430A41BC6
:1010D0001E44F6B2082E17449044E4B285F824600A
:1010E000DBD1FFF795FF0028D7D108E02B6A03EB8F
:1010F00082038342CFD0FFF78BFF0028CBD10020A3
:10110000BDE8F8830120FBE7D44D00202DE9F0472E
:101110000D46044600219046284640F27912FFF71A
:10112000A9FF234620220021284601F0A1FF231D0C
:1011300002222021284601F09BFF631D0322222169
:10114000284601F095FFA31D03222521284601F022
:101150008FFF04F1080310222821284601F088FFA0
:1011600004F1100308223821284601F081FF04F120
:10117000110308224021284601F07AFF04F11203EE
:1011800008224821284601F073FF04F114032022AD
:101190005021284601F06CFF04F118034022702111
:1011A000284601F065FF04F120030822B0212846FB
:1011B00001F05EFF04F121030822B821284601F066
:1011C00057FF04F12207C0263B4631460822284635
:1011D000083601F04DFFB6F5A07F07F10107F3D106
:1011E00004F1320308223146284601F041FF00276E
:1011F00004F1330A94F832304FEAC7099F4209F5E7
:10120000A47615D3B8F1000F08D1314604F59973CF
:101210000722284601F02CFF09F24F16274694F8C2
:1012200032213B1B93420CD3F01DC008BDE8F08770
:101230000AEB070308223146284601F019FF01375F
:10124000D8E707F2331331460822284601F010FF91
:1012500008360137E3E7000013B5044608460021CD
:1012600001602346C0F803102022019001F000FF26
:101270000198231D0222202101F0FAFE0198631D2E
:101280000322222101F0F4FE0198A31D032225214F
:1012900001F0EEFE019804F108031022282101F06C
:1012A000E7FE072002B010BDF7B50023047F0091D0
:1012B0000E4607221946054601F09EFD731C009359
:1012C000012200230721284601F096FDC4B9B31C72
:1012D0000093052223460821284601F08DFD0D24A8
:1012E0003746B278BB1B934211D32B7FA88A0734B1
:1012F000E408BBB9844294BF0020012003B0F0BDD4
:10130000AB8ADB00083BDB08B3700824E8E7FB1C72
:101310000093214600230822284601F06DFD083481
:101320000137DEE7201A18BF0120E7E7F7B50023F1
:10133000047F00910E4608221946054601F05CFD27
:10134000731CC4B90822009311462346284601F0B5
:1013500053FD1024012372785F1C013B934211D38B
:101360002B7FA88A0734E408BBB9844294BF0020CD
:10137000012003B0F0BDAB8ADB00083BDB087370D3
:101380000824E7E7F31900932146002308222846A2
:1013900001F032FD08343B46DDE7201A18BF01207A
:1013A000E7E70000F8B50E46054614460021812205
:1013B0003046FFF75FFE2B4608220021304601F041
:1013C00057FE7CB96B1C07220821304601F050FE05
:1013D0000F2401236A785F1C013B934204D3E01D74
:1013E000C008F8BD0824F4E7EB192146082230466E
:1013F00001F03EFE08343B46ECE70000F8B50E462F
:10140000054614460021CE223046FFF733FE2B4618
:1014100028220021304601F02BFE7CB905F108039B
:1014200008222821304601F023FE30242F462A7A54
:101430007B1B934204D3E01DC008F8BD2824F5E7C8
:1014400007F1090321460822304601F011FE083455
:101450000137ECE7F7B5047F00910E460123102217
:101460000021054601F0C8FCC4B9B31C0093092251
:1014700023461021284601F0BFFC19243746728804
:10148000BB1B9A4211D82B7FA88A0734E408BBB94A
:10149000844294BF0020012003B0F0BDAB8ADB0082
:1014A000103BDB0873801024E8E73B1D00932146C6
:1014B00000230822284601F09FFC08340137DEE7AC
:1014C000201A18BF0120E7E730B5094D0A449142C0
:1014D0000DD011F8013B5840082340F30004013BB4
:1014E0002C4013F0FF0384EA5000F6D1EFE730BD43
:1014F0002083B8EDF7B5384A106851686B4603C3CE
:101500006A4636493648082303F008F8044600289E
:1015100033D10A25334A106851686B4603C36A46C3
:1015200031492F48082302F0F9FF0446002849D02A
:101530000369B3F55C3F45D8B0F8661041F2B54297
:1015400091423FD1294A024402F15C018B4239D3D6
:101550005C3B234900209E1AFFF7B6FF3246074640
:1015600004F164010020FFF7AFFFA3689F4229D177
:10157000E368984208BF002524E00369B3F55C3FA7
:1015800027D8418B41F2B542914220D1174A0244FB
:1015900002F110018B4218D3103B114900209D1A13
:1015A000FFF792FF2A46064604F118010020FFF7D4
:1015B0008BFFA3689E4202D1E368984201D00D25BB
:1015C000A8E70025284603B0F0BD1025A2E70C25AA
:1015D000A0E70B259EE700BF94450008DC6F0300E1
:1015E000009000089D450008906F03000870FFF709
:1015F00010B5037C044613B9006802F077FF20465B
:1016000010BD00000023BFF35B8FC360BFF35B8F8F
:10161000BFF35B8F8360BFF35B8F7047BFF35B8F5C
:101620000068BFF35B8F704770B505460C30FFF75D
:10163000F5FF05F1080604463046FFF7EFFFA0422C
:1016400006D930466D68FFF7E9FF2544281A70BDBA
:101650003046FFF7E3FF201AF9E7000070B50546B2
:10166000406898B105F10800FFF7D8FF05F10C06B6
:1016700004463046FFF7D2FF8442304694BF6D687F
:101680000025FFF7CBFF013C2C44201A70BD000061
:1016900038B50C460546FFF7C7FFA04210D305F149
:1016A0000800FFF7BBFF04446868B4FBF0F100FBDF
:1016B0001144BFF35B8F0120AC60BFF35B8F38BD7B
:1016C0000020FCE72DE9F041144607460D46FFF7E0
:1016D000C5FF844228BF0446D4B1B84658F80C6B05
:1016E0004046FFF79BFF3044286040467E68FFF786
:1016F00095FF331A9C4203D86C600120BDE8F0814D
:101700006B60A41B3B68AB602044E8600220F5E7F7
:101710002046F3E738B50C460546FFF79FFFA04289
:1017200010D305F10C00FFF779FF04446868B4FB9F
:10173000F0F100FB1144BFF35B8F0120EC60BFF3BD
:101740005B8F38BD0020FCE72DE9FF4188466946E4
:101750000746FFF7B7FF6C4606B204EBC606002546
:10176000B44209D06268206808EB0501FFF770FCFD
:10177000636808341D44F3E729463846FFF7CAFF7B
:10178000284604B0BDE8F081F8B505460C300F4698
:10179000FFF744FF05F1080604463046FFF73EFF19
:1017A000A042304688BF6C68FFF738FF201A3860C7
:1017B00020B130462C68FFF731FF2044F8BD00000F
:1017C00073B5144606460D46FFF72EFF844228BF28
:1017D00004460190DCB101A93046FFF7D5FF019B1B
:1017E00033B93268C5E90233C5E9002401200CE0B1
:1017F0009C4238BF01942860019868608442F5D902
:101800003368AB60241AEC60022002B070BD204641
:10181000FBE700002DE9FF410F466946FFF7D0FFC7
:101820006C4600B204EBC0050026AC4209D0D4F8E7
:10183000048054F8081BB8194246FFF709FC4644D7
:10184000F3E7304604B0BDE8F081000038B5054646
:10185000FFF7E0FF044601462846FFF719FF204640
:1018600038BD00007047000010B4134602681468C9
:101870000022A4465DF8044B6047000000F580504C
:1018800090F859047047000000F5805090F8520419
:101890007047000000F5805090F958047047000030
:1018A00050207047302383F3118800F58052D2F81E
:1018B0009C34D2F898041844D2F894341844D2F8DE
:1018C0007C341844D2F88C341844D2F88834184444
:1018D000002383F31188704700F58050C0F854143A
:1018E0000120704738B5C26A936923F00103936100
:1018F000044600F04FFE0546E36A9B69DB0706D508
:1019000000F048FE431BFA2BF6D9002004E004F552
:101910008054012084F8520438BD00002DE9F04FB6
:101920000C4600F5805185B01F4691F85234BDF841
:101930003890054690469BB1D1F878340133C1F810
:1019400078342368980006D4237B082B0BD9627B5C
:101950000AB10F2B07D9D1F87C340133C1F87C349C
:101960004FF0FF3010E0302383F31188EB6AD3F897
:10197000C42012F4001B0AD0D1F880340133C1F81E
:101980008034002080F3118805B0BDE8F08FD3F8D3
:10199000C4302068C3F3014A6B6A4822002812FB56
:1019A0000A33B4BF40F080408004186022685200BF
:1019B00044BF40F000501860207B4FEA0A6242EAC0
:1019C00000425A60607B4FEA4A1610B342F440125C
:1019D0005A60D1F8B0240132C1F8B024AA1902F536
:1019E0008352117B41F020011173207B039300F09F
:1019F0002DFE039B033080105FFA8BF282420BF1C5
:101A0000010B0DDA04EB820103EB8202496891605D
:101A1000F2E7AA1902F58352117B60F34511E3E75F
:101A2000EB6A012202FA0AF2C3F8CC2005EB4A1154
:101A3000AB1903F5825301F58251C3E904871831CC
:101A4000234604F10C0253F8040B41F8040B9342B3
:101A5000F9D11B880B802E4441F2680346F803A09D
:101A600006F5805609F0030396F86C2043F0100346
:101A700022F01F02134386F86C30002383F3118891
:101A8000CDF8009042463B462146284600F0A4FD92
:101A9000012079E713B500F580540191606CFFF7E0
:101AA000DDFD1F280AD90199606C2022FFF74CFE4A
:101AB000A0F120035842584102B010BD0020FBE7BE
:101AC00008B5302383F3118800F58050406CFFF790
:101AD00099FD002383F3118808BD000000220260F5
:101AE000828142608260704710B500220023C0E905
:101AF00000230023044603810C30FFF7EFFF20464C
:101B000010BD00002DE9F0479A4688B00746884688
:101B10009146302383F3118807F580546846FFF718
:101B2000E3FF606CFFF780FD1F282DD9606C202239
:101B30006946FFF78BFE202826D194F852341BB358
:101B400003AD444605AB2E4603CE9E422060616045
:101B5000354604F10804F6D130682060B388A380CC
:101B6000DDE90023C9E90023BDF80830AAF80030F8
:101B7000002383F3118853464A464146384608B04D
:101B8000BDE8F04700F016BD002080F3118808B0D2
:101B9000BDE8F0872DE9F84F00230646C0E9013380
:101BA000284B46F8303B00F58154054688463746B9
:101BB000103438462037FFF797FFA742F9D105F5D3
:101BC00080544FF4805326630026C4E90D366764C1
:101BD000012305F5835705F5A359E66384F84030E2
:101BE00084F84830103709F110094FF0000A4FF01F
:101BF000000B47E908ABA7F11800FFF76FFF20378C
:101C000047F8286C4F45F4D184F85884A4F85A64F6
:101C1000A4F85C64A4F85E6484F86064A4F8626468
:101C2000A4F86464A4F8666484F86864B8F1000FEA
:101C300002D0054800F0A8FC044BEB622846BDE842
:101C4000F88F00BFC4450008A845000800640040A4
:101C500010B5044B197804464A1C1A70FFF79AFF16
:101C6000204610BD054E00202DE9F04300295FD02D
:101C70003048314BB3FBF1F381428CBF0A20112075
:101C8000451EB3FBF0F700FB1730ECB220B1022D7C
:101C90002846F5D8002037E07D1EB5F5806F33D299
:101CA000C4EBC40808F103034FEAE30EC3F3C70310
:101CB000A4EB030C0EF101094FF47A705FFA8CF675
:101CC0000EFB000E59FA8CFCBEFBFCFCBCF5617FE0
:101CD0001CDC1FFA8CF4581C56FA80F04743164857
:101CE000B0FBF7F7B942D5D1013BDBB20F2BD1D80E
:101CF000711EC9B207294FF0000005D81071148079
:101D00005580537191710120BDE8F08308F1FF33D4
:101D10004FEAE30CC3F3C703E41A0CF1010EE6B279
:101D20000CFB00005EFA84F4B0FBF4F4A4B2D2E73A
:101D30000846E9E73F420F000024F4000B4B10B5C2
:101D40004FF45472044600211846FFF793F9084BEC
:101D5000A3614033E361D8332362F0336362E36A03
:101D600060610022C3F8C02010BD00BF00A4004085
:101D700070A400402DE9F04F00F58055984695F885
:101D80005834012B89B004468946174604D90026E9
:101D9000304609B0BDE8F08F914A52F8231009B9D6
:101DA00042F823008F48C4F80C90017884F8108022
:101DB00099B9302383F311888B4B9A6D42F00072EE
:101DC0009A659A6B42F000729A639A6B22F00072E5
:101DD0009A630123037081F3118895F851647EB9E9
:101DE000302383F311880321152001F02DFC0321FA
:101DF000162001F029FC012385F8513486F311885F
:101E0000302383F31188E26A936923F0100393610E
:101E100000F0C0FB8246E36A9E6916F0080609D00E
:101E200000F0B8FBA0EB0A03FA2BF4D9002686F3E6
:101E30001188ADE79A6942F001029A6100F0AAFBAD
:101E40008246E36A9A69D00706D400F0A3FBA0EBB0
:101E50000A03FA2BF5D9E9E79A6942F002029A617E
:101E6000E36A4FF0000AC3F854A08AF31188686C43
:101E7000FFF7C8FB04F5825B0BF1100B2022002159
:101E80006846FFF7F7F802A8FFF728FECDF818A07C
:101E90006A460BEB06030DF1180E9446BCE80300EE
:101EA000F44518605960624603F10803F5D1DCF887
:101EB0000000186020369CF804201A71B6F5806F77
:101EC000DCD1002304F5A25285F8503485F8533450
:101ED0001A3249462046FFF7C7FE064690B9E26A25
:101EE000936923F00103936100F054FB0546E36A14
:101EF0009B69D9077FF54BAF00F04CFB431BFA2BD6
:101F0000F5D944E795F85F0495F85E24C5F86C941C
:101F1000000240EA426095F86024E36A1043B5F895
:101F20005C2440EA0240D8614FB304F5A352023268
:101F300039462046FFF798FE90B9E26A936923F08C
:101F40000103936100F026FB0546E36A9B69DA070B
:101F50007FF51DAF00F01EFB431BFA2BF5D916E7EA
:101F600095F8683495F86714C5F870741B0143EA56
:101F70000123B5F86414E26A43EA0143D3602046C2
:101F8000FFF7DCFE002385F85934E36A6FF0404226
:101F90001A65E36A154A5A65E36A44229A65E36A58
:101FA0000722C3F8DC20E36A03229045DA653FF498
:101FB000EFAEE26A936923F00103936100F0EAFA5D
:101FC0000746E36A9B69DB0705D500F0E3FAC31B0C
:101FD000FA2BF6D9DBE6012385F85234D8E600BFA8
:101FE000004E0020044E0020001002409B0008001C
:101FF0002DE9F04F054689B090469946002741F2F9
:10200000680A00F58056EB6AD3F8D430FB40D80755
:1020100051D505EB471252444FEA471B1379190774
:1020200049D4D6F884340133C6F8843405F5A55371
:10203000C3E9008913799A0648BFD6F8B43405EB92
:102040000B0248BF0133524448BFC6F8B434137979
:1020500043F008031371DB0722D596F85334FBB124
:1020600005F58254183468465C44FFF73DFD03AB28
:1020700004F1080C206861681A4603C208346445FC
:102080001346F7D120681060A2889A800123ADF82A
:1020900008302B68CDE90089DB6B694628469847F4
:1020A000D6F8A834D6F854040133C6F8A83410B1D1
:1020B00003681B6998470137202FA4D109B0BDE8F8
:1020C000F08F00002DE9F04F8DB004460F4600F070
:1020D00063FA82468946002F56D1E36AD3F89020EE
:1020E000920141BF04F58051D1F898240132C1F822
:1020F0009824D3F89020160703D100200DB0BDE836
:10210000F08FD3F89050E669C5F30125482303FB0F
:102110000566E8464046FFF7E1FC326851004ABFD9
:1021200022F06043C2F38A4343F00043920048BF69
:1021300043F080430093736813F400131FBF04F54A
:10214000805201238DF80D30D2F8B8340EBF8DF8CF
:102150000D300133C2F8B834F38803F00F038DF863
:102160000C304FF0000B9DF80C0000F06FFA5FFA96
:102170008BF3984220D9F2180CA90B44127A03F879
:102180002C2C0BF1010BEEE7012FB6D1E36AD3F84B
:102190009820950141BF04F58051D1F8982401326F
:1021A000C1F89824D3F898201007A6D0D3F89850F7
:1021B000266AC5F30125A9E7EFB9E36AC3F894508D
:1021C00004A8FFF791FC98E80F0007AD07C52B8026
:1021D0000023ADF8183023682046CDE904A9DB6B55
:1021E00004A9984704F5805458B1D4F890340133C9
:1021F000C4F8903482E7012F04BFE36AC3F89C500F
:10220000DEE7D4F894340133C4F89434012075E740
:102210002DE9F04105460F4600F580540126394668
:102220002846FFF74FFF10B184F85364F7E7D4F85E
:10223000A834D4F854040133C4F8A83420B1036896
:10224000BDE8F0411B691847BDE8F081F0B5C36AED
:102250001A6C12F47F0F2BD000F580541B6CC4F85D
:10226000AC3441F26805002347194FF0010C00EB34
:1022700043122A445E01117911F0020F15D049076B
:1022800013D4B959C66AD6F8C8E00CFA01F111EABC
:102290000E0F0AD0C6F8D010117941F00401117167
:1022A000D4F88C240132C4F88C240133202BDED1E5
:1022B000F0BD000010B5254C254B226802B338B3A1
:1022C0001A6D12060ED580221A6500F065F950EAE3
:1022D00001020B4602D0013861F10003024620687A
:1022E000FFF786FE1A4A136D1B032AD523684FF4A5
:1022F000002103F580531165012283F8592420E061
:1023000001221A6508221A654FF480621A6510BD11
:10231000196DC80702D4196D890705D50321196500
:1023200010460021FFF774FF094B1A6D100702D405
:102330001A6DD10605D518221A6520680121FFF70C
:1023400067FF2068BDE81040FFF780BF004E002007
:102350000064004008B5302383F31188FFF776FF4F
:10236000002383F3118808BDC36AD3F8C40080F446
:102370000010C0F34050704708B5302383F3118834
:1023800000F58050406CFFF74FF9002383F311886C
:1023900043090CBF0120002008BD000000F5805358
:1023A00093F8592462B1C16A8A6922F001028A61F4
:1023B000D3F89C240132C3F89C24002283F85924CA
:1023C000704700002DE9F743302181F3118800F5B3
:1023D00082511031002541F2680E4FF0010800F5DE
:1023E000805C00EB45147444267977071CD4F6060C
:1023F0001AD5D0F82C908E69D9F8C87008FA06F66C
:102400003E4211D04F6801970F689742019F9F414C
:102410000AD2C9F8D060267946F004062671DCF8A5
:1024200088440134CCF888440135202D01F1200185
:10243000D7D1002383F3118803B0BDE8F0830000F7
:10244000F8B51E46002313700F4605461446FFF7E5
:1024500093FF80F0010038701EB12846FFF784FF1B
:102460002070F8BD2DE9F04F85B09946DDE90EA347
:102470000D4602931378019391F800B080461646FA
:1024800000F08AF82B7804460F4613B93378002BF6
:1024900041D022463B464046FFF794FFFFF75AFFE4
:1024A000FFF77CFF4B4632462946FFF7C9FF2B78E2
:1024B00033B1BBF1000F03D0012005B0BDE8F08FB0
:1024C000337813B1019B002BF6D108F580530393A9
:1024D000029B544577EB03031DD2039BD3F85404AE
:1024E000C8B10368AAEB04011B6898474B46324603
:1024F00029464046FFF7A4FF2B7813B1BBF1000F2C
:10250000DAD1337813B1019B002BD5D100F044F818
:1025100004460F46DCE70020CFE7000008B50020A6
:10252000FFF7C8FEBDE8084001F050B808B501202B
:10253000FFF7C0FEBDE8084001F048B800B59BB009
:10254000EFF3098168226846FEF782FDEFF3058309
:10255000014B9B6BFEE700BF00ED00E008B5FFF705
:10256000EDFF000000B59BB0EFF3098168226846DB
:10257000FEF76EFDEFF30583014B5B6BFEE700BFDB
:1025800000ED00E0FEE700000FB408B5029801F08E
:102590000FF9FEE701F0EEBB01F0D0BB13B56C46BE
:1025A00084E80600031D94E8030083E80500012089
:1025B00002B010BD73B58568019155B11B885B07EA
:1025C00007D4D0E900369B6B9847019AC1B23046D8
:1025D000A847012002B070BDF0B5866889B00546F5
:1025E0000C465EB1BDF838305B070AD4D0E900373D
:1025F0009B6B98472246C1B23846B047012009B0CC
:10260000F0BD00220023CDE900230023ADF80830FF
:102610000A4603AB01F10806106851681C4603C462
:102620000832B2422346F7D1106820609288A28017
:10263000FFF7B2FF0423ADF808302B68CDE90001A5
:10264000DB6B694628469847D8E70000082817D969
:1026500009280CD00A280CD00B280CD00C280CD040
:102660000D280CD00E2814BF4020302070470C20BD
:1026700070471020704714207047182070472020A2
:10268000704700002DE9F041456A15B94162BDE887
:10269000F0814B6823F06047C3F38A464FEAD37E4C
:1026A000C3F3807816EA230638BF3E46AC462B4675
:1026B0005A68BEEBD27F22F060440AD0002A18DAB2
:1026C000A40CB44217D19D420FD10D60DEE7134632
:1026D000EEE7A74207D102F08044C2F38072424580
:1026E0000BD054B1EFE708D2EDE7CCF800100B6047
:1026F000CDE7B44201D0B442E5D81A689C46002A1E
:10270000E5D11960C3E700002DE9F047089D01F00D
:1027100007044FEAD508224405F0070500EBD10075
:102720004FF47F49944201D1BDE8F08704F00707D8
:1027300005F0070A57453E4638BF5646C6F108061B
:10274000111B8E4228BF0E46E10808EBD50E415CF6
:1027500013F80EC0B94029FA06F721FA0AF1FFB2C0
:102760008CEA010147FA0AF739408CEA010C03F8B8
:102770000EC034443544D5E780EA0120082341F2F5
:10278000210201B24000002980B203F1FF33B8BF3B
:10279000504013F0FF03F4D17047000038B50C46E9
:1027A0008D18A54200D138BD14F8011BFFF7E4FFD6
:1027B000F7E7000042684AB11368436043898189A2
:1027C00001339BB29942438138BF838110467047E1
:1027D00070B588B0202204460D4668460021FEF7F9
:1027E00049FC20460495FFF7E5FF024658B16B46C9
:1027F000054608AE1C4603CCB442286069602346F7
:1028000005F10805F6D1104608B070BD082817D9A3
:1028100009280CD00A280CD00B280CD00C280CD07E
:102820000D280CD00E2814BF4020302070470C20FB
:1028300070471020704714207047182070472020E0
:1028400070470000082817D90C280CD910280CD97B
:1028500014280CD918280CD920280CD930288CBF62
:102860000F200E207047092070470A2070470B2068
:1028700070470C2070470D20704700002DE9F84389
:10288000078C072F04461ED9D0E9029800254FF681
:10289000FF73C5F12006A5F1200029FA05F108FA19
:1028A00006F628FA00F031430143C9B21846FFF793
:1028B00063FF0835402D0346EBD1E1693A46BDE898
:1028C000F843FFF76BBF4FF6FF70BDE8F8830000D9
:1028D00010B54B6823B9CA8A63F30902CA8210BDD6
:1028E00004691A681C600361C38A013BC3824A60A1
:1028F000EFE700002DE9F84F1D46CB8A0F46C3F3E2
:1029000009010529814692460B4630D00020AAB223
:1029100007F11A049EB2042E1FFA80F80FD89045D2
:1029200003F1010306D3FB8A0A4462F30903FB8225
:1029300001201AE01AF80060E6540130EAE79045F9
:10294000F1D2A1F1050B1C237C68BBFBF3F203FB66
:1029500012BB1FFA8BF6002C45D14846FFF72AFF21
:10296000044638B978606FF00200BDE8F88F4FF088
:102970000008E6E7002606607860ADB24FF0000B75
:10298000454510D90AEB0803221D13F8011B915588
:10299000B1B208F101081B291FFA88F82BD0454570
:1029A00006F10106F1D8FB8AC3F30902154465F369
:1029B0000903BCE7013292B21C462368002BF9D10F
:1029C0006B1F0B441C21B3FBF1F301339BB29A4202
:1029D000D3D2BBF1000FD0D14846FFF7EBFE20B9B0
:1029E000C4F800B0BFE70122E7E7C0F800B05E46D8
:1029F00020600446C1E74545D5D94846FFF7DAFED1
:102A000008B92060AFE7C0F800B000262060044697
:102A1000B6E700002DE9F04F2DED028B1C4683B088
:102A20005B69019207468846002B00F09A80238C50
:102A30002BB1E269002A00F09480072B35D807F10A
:102A40000C00FFF7B7FE054638B96FF002052846BF
:102A500003B0BDEC028BBDE8F08F14220021FEF71D
:102A600009FB228CE16905F10800FEF7F1FA208CE0
:102A7000013080B2FFF7E6FEFFF7C8FE013880B2F2
:102A80002084013028746369228C1B782A4403F067
:102A90001F0363F03F0348F000411372384669603A
:102AA0002946FFF7EFFD0125D1E700F10C034FF0B8
:102AB000000908EE103A4FF0800A4E464D4618EED7
:102AC000100AFFF777FE83460028BED014220021AB
:102AD000FEF7D0FA002E3AD1019BABF80830022263
:102AE0000BF1080E1FFA82FC0CF10100BCF1060F7D
:102AF000218C80B201D88E422BD3FFF7A3FEFFF7C3
:102B000085FE62691278013802F01F028E4208BF0A
:102B10004FF0400A42EA49121BFA80F14AEA020ADF
:102B2000013048F0004281F808A08BF81000CBF883
:102B3000042059463846FFF7A5FD238C0135B342E2
:102B40002DB289F001094FF0000AB8D17FE70022C9
:102B5000C6E7E169895D0EF802100136B6B20132AE
:102B6000C0E76FF0010572E7F8B515460E46302252
:102B7000002104461F46FEF77DFA069B6360B5F50B
:102B8000001F079BA76034BF6A094FF6FF72A3625C
:102B900097B2E66104F1100000239A4206D80023A0
:102BA0000360A782E3822383E360F8BD06600133FC
:102BB00030462036F1E7000003781BB94BB2002BFA
:102BC000C8BF01707047000000787047F8B50C4628
:102BD000C969074611B9238C002B37D1257E1F2DDB
:102BE00034D8387828BB228C072A2CD8268A36F08D
:102BF00003032BD14FF6FF70FFF7D0FD20F001004B
:102C00003102400441EA0561400C41EA40254FF69B
:102C1000FF72234629463846FFF7FCFE002807DDF1
:102C2000626913780133DBB21F2B88BF0023137056
:102C3000F8BD218A2D0645EA012505432046FFF708
:102C40001DFE0246E5E76FF00300F1E76FF00100BB
:102C5000EEE7000070B58AB004461646002128222F
:102C600068461D46FEF706FABDF83830ADF810305C
:102C70000F9B05939DF840308DF81830119B0793FA
:102C80006946BDF84830ADF820302046CDE90265F0
:102C9000FFF79CFF0AB070BD2DE9F041D3690546EE
:102CA0000C4616460BB9138C5BBB377E1F2F28D8FA
:102CB00095F80080B8F1000F26D03046FFF7DEFD12
:102CC0003378210241EAC33141EA0801338A41EAFB
:102CD000076141EA03410246334641F0800128463C
:102CE000FFF798FE00280ADD3378012B07D17269BF
:102CF00013780133DBB21F2B88BF00231370BDE8AC
:102D0000F0816FF00100FAE76FF00300F7E70000D1
:102D1000F0B58BB004460D461746002128226846C0
:102D20001E46FEF7A7F99DF84C305A1E53425341F8
:102D30008DF800309DF84030ADF81030119B0593B0
:102D40009DF848308DF81830149B07936A46BDF8FB
:102D50005430ADF8203029462046CDE90276FFF701
:102D60009BFF0BB0F0BD0000406A00B1043070471B
:102D7000436A1A68426202691A600361C38A013BAE
:102D8000C38270472DE9F041D0F82080194E1446D7
:102D90001D464146002709B9BDE8F081D1E902236B
:102DA000A21A65EB0303964277EB03031ED2036A74
:102DB0008B420DD1FFF78CFD036A1B680362036928
:102DC0000B60C38A0161016A013BC3828846E2E766
:102DD000FFF77EFD0B68C8F8003003690B60C38AFB
:102DE0000161013BC382D8F80010D4E78846096826
:102DF000D1E700BF80841E002DE9F04F8BB00D4657
:102E0000DDF8509014469B468046002800F019815A
:102E1000B9F1000F00F01581531E3F2B00F2118114
:102E2000012A03D1BBF1000F40F00B810023CDE953
:102E30000833B8F81430B5EBC30F4FEAC30703D318
:102E400000200BB0BDE8F08F2B199F42D8F80C3052
:102E50003ABF7F1BFFB227461BB9D8F81030002BB2
:102E60007AD0272D4ED8C5F12806B7424FF000037F
:102E70002CBFF6B23E4600932946D8F8080008ABAE
:102E80003246FFF741FCA7EB060A35445FFA8AFA9F
:102E9000B8F8143003F10053053BDB000493D8F875
:102EA0000C3003932821039B13B1BAF1000F2CD1EE
:102EB000D8F8100040B1BAF1000F05D0009608AB69
:102EC0005246691AFFF720FC38B2002FB8D06607C7
:102ED0000AD00AAB03EBD401624211F8083C02F0BD
:102EE0000702134101F8083C082C3CD9102C40F291
:102EF000B580202C40F2B780BBF1000F00F09C8021
:102F0000082334E0BA460026C2E7049BE02B28BF22
:102F1000E02306930B44AB42059314D95A1B039844
:102F20000096924534BF5246D2B2691A08AB0430BB
:102F30000792FFF7E9FB079A1644AAEB020A154429
:102F4000F6B25FFA8AFA049B069A05999B1A0493D3
:102F5000039B1B680393A6E70093D8F8080008AB0F
:102F60003A462946AEE7BBF1000F13D00123B4EB7C
:102F7000C30F6CD0082C12D89DF82030621E23FAA3
:102F800002F2D50706D54FF0FF3202FA04F42343CC
:102F90008DF820309DF8203089F8003051E7102C52
:102FA00012D8BDF82030621E23FA02F2D10706D5EE
:102FB0004FF0FF3202FA04F42343ADF82030BDF89D
:102FC0002030A9F800303CE7202C0FD80899631E68
:102FD00021FA03F3DA0705D54FF0FF3202FA04F4C1
:102FE0000C430894089BC9F800302AE7402C2BD0EA
:102FF000DDE90865611EC4F12102A4F1210326FA6E
:1030000001F105FA02F225FA03F311431943CB0744
:1030100012D50122A4F12003C4F1200102FA03F326
:1030200022FA01F1A240524243EA010363EB430357
:1030300032432B43CDE90823DDE90823C9E9002306
:10304000FFE66FF00100FCE66FF00800F9E6082CDF
:10305000A0D9102CB3D9202CEED8C3E7BBF1000FB8
:10306000ADD0022383E7BBF1000FBBD004237EE782
:1030700030B5012A144638BF0124402C85B028BF42
:1030800040240025012ACDE9025518D81B788DF877
:10309000083063070AD004AB03EBD405624215F88D
:1030A000083C02F00702934005F8083C00910346F3
:1030B0002246002102A8FFF727FB05B030BD082AF1
:1030C000E4D9102A03D81B88ADF80830E1E7202A9C
:1030D0008DBFD3E900231B680293CDE90223D8E713
:1030E00010B5CB681BB98B600B618B8210BD046976
:1030F0001A681C600361C38A013BC382CA60F0E79F
:1031000003064CBFC0F3C0300220704708B502462A
:10311000FFF7F6FF022806D15306C2F30F2001D1B4
:1031200000F0030008BDC2F30740FBE72DE9F04FB4
:1031300093B0CDE903230A6804461046FFF7E0FF89
:10314000022814BFC2F306260026002A0D46824636
:1031500080F2F28112F0C04940F0EE81097B002933
:1031600000F0EA81022803D02378B34240F0E781DF
:10317000C2F304630693104602F07F030593FFF742
:10318000C5FF059B29444FEA834848EA0A4848EAB4
:103190004668CE7800230022CDE90823F309834650
:1031A00048EA0008029367D0059B009302466768CF
:1031B000534608A92046B847002800F0C381276A73
:1031C0004FB9414604F10C00FFF702FB074690B9E6
:1031D0006FF0020054E03B6998450DD03F68002F26
:1031E000F9D1414604F10C00FFF7F2FA0746002836
:1031F000EED0236A3B60276297F817C006F01F08DD
:10320000CCF3840CACEB08001FFA80FE0028B8BF9A
:103210000EF12000A8EB0C031FFA83FED7E9022170
:10322000B8BF00B2002B0793BEBF0EF120031BB244
:10323000079352EA010338D0039BDFF824E39A1A7C
:10324000049B4FF0000C63EB010196457CEB0103FE
:103250002BD36B7B97F81AE0734519D1029B002B97
:1032600078D0012821DC7868F8B9DFF8F0C29445FD
:1032700070EB010316D337E0276A27B96FF00C0013
:1032800013B0BDE8F08F3B699845B5D03F68F4E7CF
:10329000B24890427CEB010301D30020F0E7029B8F
:1032A000002BFAD0079B0F2B17DCFA7DB30002F03E
:1032B000030203F07C031343FB7539462046FFF7F6
:1032C00007FB6B7BBB76029B3BB9FB7DC3F38402A0
:1032D000013262F38603FB75D0E76A7BBB7E9A42BC
:1032E000DBD1029B002B35D0B309022B32D0039BDC
:1032F000BB60049BFB60142200210DA8FDF7BAFE01
:10330000039B0A93049B0B932B1D0C932B7BADF813
:103310003EB0013BDBB2ADF83C30069B8DF842304D
:10332000059B8DF8433094F82C308DF840A083F045
:1033300001038DF844308DF84180A3680AA9204626
:103340009847FB7DC3F38403013303F01F039B0203
:10335000FB82A2E7FB7DC6F34012B2EBD31F40F025
:10336000F480C3F38403434540F0F280029A2B7B40
:10337000B609002A4DD0F2075DD4032B40F2EB8052
:10338000039BBB60049BFB602B7BAE1D033BDBB24E
:103390003246394604F10C00FFF7ACFA00280CDA8B
:1033A00039462046FFF794FAFB7DC3F384030133CB
:1033B00003F01F039B02FB820AE7DDE90884AB8868
:1033C0003B834FF6FF73C9F12000A9F1200228FAD0
:1033D00009F104FA00F0014324FA02F211431846FD
:1033E000C9B2FFF7C9F909F10809B9F1400F03465D
:1033F000E9D1B8822A7B033AD2B23146FFF7CEF93F
:10340000FB7DB882DA43C2F3C01262F3C713FB75C7
:1034100043E786B92E1D013BDBB23246394604F143
:103420000C00FFF767FA0028BADB2A7BB88A013A5A
:10343000D2B23146E2E7F98AC1F30901013B04291E
:10344000DAB25BD8281D002307F11B069A4208D97F
:1034500010F801CB06F801C0013101330529DBB2B8
:10346000F4D103990A9104990B91934207F11B013E
:103470000C9138BF043379680D9134BF55FA83F34A
:1034800000230E93FB8AADF83EB0C3F309031A4440
:10349000069B8DF84230059B8DF8433094F82C3014
:1034A000ADF83C2083F001038DF8443000238DF803
:1034B00040A08DF841807B602A7BB88A013A291DA3
:1034C000FFF76CF93B8BB882834203D1A3680AA94A
:1034D0002046984720460AA9FFF702FEFB7DBA8ADC
:1034E000C3F38403013303F01F039B02FB823B8B76
:1034F0009A420CBF00206FF01000C1E67B68002BE1
:10350000AFD0052001E01C3033461E68002EFAD1F2
:10351000091A081D2E1D184401EB090CBCF11B0FE4
:103520005FFA89F39DD89A429BD916F8013B00F8BF
:10353000013B09F10109EFE76FF00900A0E66FF028
:103540000A009DE66FF00B009AE66FF00D0097E61B
:103550006FF00E0094E66FF00F0091E640420F000E
:1035600080841E00EFF3098305494A6B22F00102B3
:103570004A63683383F30988002383F31188704713
:1035800000EF00E0302080F3118862B60C4B0D4A4A
:10359000D96821F4E0610904090C0A43DA60D3F820
:1035A000FC20094942F08072C3F8FC200A6842F00E
:1035B00001020A602022DA7783F82200704700BFF8
:1035C00000ED00E00003FA05001000E010B5302324
:1035D00083F311880E4B5B6813F4006314D0F1EE93
:1035E000103AEFF30984683C4FF08073E361094BB4
:1035F000DB6B236684F3098800F0A4F810B1064B56
:10360000A36110BD054BFBE783F31188F9E700BF09
:1036100000ED00E000EF00E03F0300084203000877
:103620004FF0E023002258684FF0FF31930003F180
:10363000604303F5614301329042C3F88010C3F840
:103640008011F3D27047000000F1604303F561433D
:103650000901C9B283F80013012200F01F039A4048
:1036600043099B0003F1604303F56143C3F88021E4
:103670001A60704700230375826803691B689968A4
:103680009142FBD25A6803604260106058607047F4
:1036900000230375826803691B6899689142FBD80F
:1036A0005A680360426010605860704708B5084669
:1036B000302383F311880B7D032B05D0042B0DD011
:1036C0002BB983F3118808BD8B6900221A604FF073
:1036D000FF338361FFF7CEFF0023F2E7D1E9003229
:1036E00013605A60F3E70000FFF7C4BF054BD968C9
:1036F0000875186802681A60536001220275D86064
:10370000FCF708BE104E002030B50C4BDD684B1C9A
:1037100087B004460FD02B46094A684600F02AF9C4
:103720002046FFF7E3FF009B13B1684600F02CF939
:10373000A86907B030BDFFF7D9FFF9E7104E0020A8
:10374000AD360008044B1A68DB6890689B689842A5
:1037500094BF002001207047104E0020084B10B588
:103760001C68D86822681A60536001222275DC60E8
:10377000FFF78EFF01462046BDE81040FCF7CABDAA
:10378000104E002038B5074C074908480123002592
:103790002370656000F0ECFB0223237085F3118831
:1037A00038BD00BF7850002008460008104E0020A9
:1037B00008B572B6044B186500F0ACFA00F05AFB7D
:1037C000024B03221A70FEE7104E002078500020B2
:1037D00000F010B98B60022308618B8208467047A5
:1037E0008368A3F1840243F8142C026943F8442C43
:1037F000426943F8402C094A43F8242CC26843F834
:10380000182C022203F80C2C002203F80B2C044A7B
:1038100043F8102CA3F12000704700BF2D030008CF
:10382000104E002008B5FFF7DBFFBDE80840FFF7AA
:103830005BBF0000024BDB6898610F20FFF756BFAB
:10384000104E0020302383F31188FFF7F3BF0000F0
:1038500008B50146302383F311880820FFF754FF91
:10386000002383F3118808BD10B503689C68A24249
:103870000CD85C688A600B604C6021605960996864
:103880008A1A9A604FF0FF33836010BD1B68121BC9
:10389000ECE700000A2938BF0A2170B504460D463E
:1038A0000A26601900F05EFB00F04AFB041BA542EB
:1038B00003D8751C2E460446F3E70A2E04D9BDE84A
:1038C0007040012000F094BB70BD0000F8B5144BAF
:1038D0000D46D96103F1100141600A2A196982601D
:1038E00038BF0A22016048601861A818144600F029
:1038F0002BFB0A2700F024FB431BA342064606D3FA
:103900007C1C281900F02EFB27463546F2E70A2FCB
:1039100004D9BDE8F840012000F06ABBF8BD00BF43
:10392000104E0020F8B506460D4600F009FB0F4A80
:10393000134653F8107F9F4206D12A46014630466F
:10394000BDE8F840FFF7C2BFD169BB68441A2C1923
:1039500028BF2C46A34202D92946FFF79BFF2246E7
:1039600031460348BDE8F840FFF77EBF104E002007
:10397000204E002010B4C0E9032300235DF8044B5F
:103980004361FFF7CFBF000010B5194C236998427F
:103990000DD0D0E90032816813605A609A680A44F9
:1039A0009A60002303604FF0FF33A36110BD2346EC
:1039B000026843F8102F53600022026022699A4285
:1039C00003D1BDE8104000F0C7BA936881680B448A
:1039D000936000F0B5FA2269E1699268441AA24244
:1039E000E4D91144BDE81040091AFFF753BF00BFE6
:1039F000104E00202DE9F047DFF8BC8008F11007D9
:103A00002C4ED8F8105000F09BFAD8F81C40AA6849
:103A1000031B9A423ED81444D5E900324FF0000906
:103A2000C8F81C4013605A60C5F80090D8F81030F0
:103A3000B34201D100F090FA89F31188D5E903313E
:103A400028469847302383F311886B69002BD8D020
:103A500000F076FA6A69A0EB04094A4582460DD265
:103A6000022000F0C5FA0022D8F81030B34208D185
:103A700051462846BDE8F047FFF728BF121A2244F6
:103A8000F2E712EB090938BF4A4629463846FFF7E4
:103A9000EBFEB5E7D8F81030B34208D01444211A31
:103AA000C8F81C00A960BDE8F047FFF7F3BEBDE809
:103AB000F08700BF204E0020104E002038B500F0E7
:103AC0003FFA054AD2E90845031B181945F10001E0
:103AD000C2E9080138BD00BF104E00200020704729
:103AE000FEE70000704700004FF0FF307047000015
:103AF000BFF34F8F024A1369DB03FCD4704700BF4A
:103B00000020024008B5094B1B7873B9FFF7F0FF9E
:103B1000074B5A69002ABFBF064A9A6002F18832F1
:103B20009A601A6822F480621A6008BD90500020E2
:103B3000002002402301674508B50B4B1B7893B961
:103B4000FFF7D6FF094B5A6942F000425A611A68E2
:103B500042F480521A601A6822F480521A601A687D
:103B600042F480621A6008BD90500020002002409C
:103B70007F289ABF00F58030C00200207047000007
:103B80004FF4006070470000802070477F2808B520
:103B90000BD8FFF7EDFF00F500630268013204D196
:103BA00004308342F9D1012008BD0020FCE7000069
:103BB0007F2810B504461FD8FFF79AFFFFF7A2FF32
:103BC0000E4BF3221A6102225A615A6942EAC0027C
:103BD0005A615A6942F480325A61FFF789FF4FF403
:103BE0000061FFF7C5FF00F041F9FFF7A5FF204690
:103BF000BDE81040FFF7CABF002010BD0020024002
:103C00002DE9F84340EA020313F00703144606D0F7
:103C1000304B40F233321A600020BDE8F88385183B
:103C20002D4A95420CD92B4A4FF44E711160F3E79F
:103C3000031D1B684A68934208D1083C08300831CC
:103C4000072C14D902680B689A42F1D0FFF75AFF8B
:103C5000FFF74EFF214E08314FF001084FF00009E9
:103C6000012CA1F1080706D8FFF766FF01E0002C40
:103C7000ECD10120D1E7C6F81480054651F8083C84
:103C800045F8043B51F8043C4360FFF731FF3369CA
:103C900043F001033361C6F81490026851F8083C00
:103CA0009A420CD00B4B4FF458721A600C4B1860B0
:103CB0000C4B1C600C4B1F60FFF73EFFACE72D6800
:103CC00051F8043C9D4201F10801EBD1083C083059
:103CD000C6E700BF8C50002000000408002002400E
:103CE000805000208850002084500020084908B5EA
:103CF0000B7828B11BB9FFF705FF01230B7008BD36
:103D0000002BFCD0BDE808400870FFF715BF00BFCE
:103D10009050002008B54FF4C0314FF0005000F033
:103D2000A7F8BDE808404FF480414FF0805000F004
:103D30009FB80000084600F0D9BB000038B5EFF38B
:103D400011859DB9EFF30584C4F30804302334B121
:103D500083F31188FFF7B2FE85F3118838BD83F332
:103D60001188FFF7ABFE84F3118838BDBDE83840F9
:103D7000FFF7A4BE38B5FFF7E1FF114C114AC008A8
:103D800040EA4170A0FB025EC908A0FB040C1CEBDA
:103D9000050CA1FB04404FF000035B41A1FB0212A4
:103DA0001CEB040C43EB000011EB0E0142F100028E
:103DB000411842F10000090941EA007038BD00BF16
:103DC000CFF753E3A59BC4200244D2B2904200D166
:103DD0007047431C800000F1804000F514500068DB
:103DE00041F8040BD8B2F1E7124B10B5D3F890406C
:103DF000240409D4D3F89040C3F89040D3F89040FD
:103E000044F40044C3F890400B4C2368024443F44C
:103E100080732360D2B2904200D110BD431C800059
:103E200000F1804000F5145051F8044B0460D8B202
:103E3000F1E700BF001002400070004007B501220A
:103E400001A90020FFF7C0FF019803B05DF804FB53
:103E500013B50446FFF7F2FFA04205D0012201A9E5
:103E600000200194FFF7C0FF02B010BD70470000B2
:103E70007047000070470000074B45F255521A602A
:103E800002225A6040F6FF729A604CF6CC421A60E9
:103E9000024B01221A7070470030004098500020F9
:103EA000034B1B781BB1034B4AF6AA221A607047DA
:103EB0009850002000300040054B1A6832B902F1DA
:103EC000804202F50432D2F894201A60704700BF95
:103ED00094500020024B4FF40002C3F89420704726
:103EE0000010024008B5FFF7E7FF024B1868C0F367
:103EF000407008BD9450002070470000FEE70000AD
:103F00000A4B0B480B4A90420BD30B4BDA1C121A8C
:103F1000C11E22F003028B4238BF00220021FDF7B0
:103F2000A9B853F8041B40F8041BECE764470008E9
:103F30001C5100201C5100201C51002000F0C2B870
:103F40004FF08043586A70474FF080430022586317
:103F50001A610222DA6070474FF080430022DA6073
:103F6000704700004FF0804358637047FEE7000041
:103F700070B51B4B01630025044686B0586085620E
:103F80000E46FFF7FFFA04F11003C4E904334FF0C3
:103F9000FF33C4E90635C4E90044A560E562FFF7D4
:103FA000CFFF2B460246C4E9082304F134010D4A31
:103FB000256580232046FFF70DFC0123E0600A4AB7
:103FC0000375009272680192B268CDE90223074B33
:103FD0006846CDE90435FFF725FC06B070BD00BF8B
:103FE0007850002014460008194600086D3F00086C
:103FF000024AD36A1843D062704700BF104E0020B7
:104000004B6843608B688360CB68C3600B69436116
:104010004B6903628B6943620B6803607047000061
:1040200008B5204BDA6A42F07F02DA62DA6A22F0DF
:104030007F02DA62DA6ADA6C42F07F02DA64DA6E00
:1040400042F07F02DA66184ADB6E11464FF090406C
:10405000FFF7D6FF02F11C0100F58060FFF7D0FFEB
:1040600002F1380100F58060FFF7CAFF02F1540148
:1040700000F58060FFF7C4FF02F1700100F5806079
:10408000FFF7BEFF02F18C0100F58060FFF7B8FF7B
:1040900002F1A80100F58060FFF7B2FFBDE808401B
:1040A00000F050B8001002402046000808B500F0AB
:1040B000EDF9FFF767FBBDE80840FFF7FDBE000024
:1040C000704700000F4B9A6D42F001029A659A6F9B
:1040D00042F001029A670C4A9B6F936843F0010318
:1040E00093604FF08043A7229A624FF0FF32DA626A
:1040F00000229A615A63DA605A6001225A611A609A
:10410000704700BF00100240002004E04FF08042E2
:1041100008B51169D3680B40D9B2C9439B07116137
:1041200007D5302383F31188FFF752FB002383F375
:10413000118808BD08B5FFF773FABDE8084000F024
:1041400081B900004E4B4FF0FF319A6A99629A6A2A
:1041500000229A62986AD86A60F07F00D862D86AB2
:1041600000F07F00D862D86A186B1963186B1A6365
:10417000186B986B9963986B9A63986BD86BD9633B
:10418000D86BDA63D86B186C1964196C1A64196CE3
:10419000196E41F001011966D3F8801021F0010178
:1041A000C3F88010D3F88010996D41F08051996563
:1041B000996F21F080519967996F32494FF400400F
:1041C0008860CA600A624A628A62CA620A634A6393
:1041D0008A63CA630A644A648A64CA640A654A656F
:1041E0004A604FF48072C1F880204FF440720A6038
:1041F0004A6912F48062FBD1D3F8901011F4407F29
:104200001EBF4FF48031C3F89010C3F89020D3F84C
:10421000982042F00102C3F89820D3F89820920722
:10422000FBD51A6842F480321A601A689003FCD5F4
:10423000D3F8902022F00322C3F89020124ADA60CB
:104240001A6842F080721A601A689101FCD50F4911
:104250000F4800229A60C3F888100E49C3F89C20CA
:10426000016002684A401207FBD19A6842F00302DB
:104270009A609A6802F00C020C2AFAD1704700BFCB
:104280000010024000700040132A610155010050E7
:104290000020024004070400074A08B5536903F0F0
:1042A0000103536123B1054A13680BB15068984765
:1042B000BDE80840FFF78AB9000401409C50002087
:1042C000074A08B5536903F00203536123B1054A55
:1042D00093680BB1D0689847BDE80840FFF776B9FE
:1042E000000401409C500020074A08B5536903F0C0
:1042F0000403536123B1054A13690BB15069984710
:10430000BDE80840FFF762B9000401409C5000205E
:10431000074A08B5536903F00803536123B1054AFE
:1043200093690BB1D0699847BDE80840FFF74EB9D3
:10433000000401409C500020074A08B5536903F06F
:104340001003536123B1054A136A0BB1506A9847B1
:10435000BDE80840FFF73AB9000401409C50002036
:10436000164B10B55C6904F478725A61A30604D543
:10437000134A936A0BB1D06A9847600604D5104A75
:10438000136B0BB1506B9847210604D50C4A936B05
:104390000BB1D06B9847E20504D5094A136C0BB1F9
:1043A000506C9847A30504D5054A936C0BB1D06CAB
:1043B0009847BDE81040FFF709B900BF000401406D
:1043C0009C500020194B10B55C6904F47C425A6182
:1043D000620504D5164A136D0BB1506D984723053D
:1043E00004D5134A936D0BB1D06D9847E00404D502
:1043F0000F4A136E0BB1506E9847A10404D50C4AB6
:10440000936E0BB1D06E9847620404D5084A136FBF
:104410000BB1506F9847230404D5054A936F0BB135
:10442000D06F9847BDE81040FFF7D0B800040140B6
:104430009C50002008B5FFF769FEBDE80840FFF773
:10444000C5B80000062108B50846FFF7FDF80621AB
:104450000720FFF7F9F806210820FFF7F5F80621F5
:104460000920FFF7F1F806210A20FFF7EDF80621F1
:104470001720FFF7E9F806212820FFF7E5F8BDE847
:10448000084007211C20FFF7DFB8000008B5FFF740
:1044900051FE00F007F8FFF713FEBDE80840FFF7F4
:1044A0004DBD00000023054A19460133102BC2E917
:1044B000001102F10802F8D1704700BF9C500020A3
:1044C0000B460146184600F003B8000000F00EB895
:1044D00010B5054C13462CB10A4601460220AFF335
:1044E000008010BD2046FCE700000000024B0146A2
:1044F0001868FFF71FBC00BF1823002010B5013952
:104500000244904201D1002005E0037811F8014FE8
:10451000A34201D0181B10BD0130F2E72DE9F04194
:10452000A3B1C91A17780144044603F1FF3C8C4239
:10453000204601D9002009E00578BD4204F10104BC
:10454000F5D10CEB0405D618A54201D1BDE8F081E8
:1045500015F8018D16F801EDF045F5D0E7E70000FC
:10456000034611F8012B03F8012B002AF9D17047FB
:10457000696E2E7369657272616165726F737061C5
:1045800063652E547275654E617650726F2D473497
:104590000000000040A2E4F1646891060041A3E538
:1045A000F2656992070000004261642043414E4970
:1045B0006661636520696E6465782E000000000006
:1045C00000000000751D0008691800086524000837
:1045D000D91800081D190008051B0008E518000877
:1045E000A1180008A51800087D1800086518000823
:1045F000C11A0008891800089D25000895180008B0
:10460000951A00086330000004460008684E002038
:10461000785000206D61696E0069646C650000006F
:104620000001942A00000000AAAAAAAA00001424EB
:10463000FFFF0000000000000090090000040000DF
:1046400000000000AAA6AAAA00000000DFFF0000E8
:10465000000000000000000000000000000000005A
:10466000AAAAAAAA00000000FFFF000000000000A4
:10467000000000000000000000000000AAAAAAAA92
:1046800000000000FFFF000000000000000000002C
:104690000000000000000000AAAAAAAA0000000072
:1046A000FFFF00000000000000000000000000000C
:1046B00000000000AAAAAAAA00000000FFFF000054
:1046C00000000000000000000000000000000000EA
:1046D000AAAAAAAA00000000FFFF00000000000034
:1046E0000000000000000000B51400000000000001
:1046F0000070030000000000FE2A0100D204000048
:104700001C2300200000000000000000000000004A
:104710000000000000000000000000000000000099
:104720000000000000000000000000000000000089
:104730000000000000000000000000000000000079
:104740000000000000000000000000000000000069
:104750000000000000000000000000000000000059
:044760000000000055
:00000001FF
